:105D4A0001130000770101030200000301FA0400B5
:105D5A00FA0500030A0A5A0B001E0C00FA0D00038A
:105D6A000E00030F0164100096120132130AFA148E
:105D7A00020215000017010A1801FA1905321A0160
:105D8A000A1B01FA1C05321FFFFF20FFFF23011E19
:105D9A002400642A00FA2B00FA2C50782D003C2E9D
:105DAA0000462F001E3000643250783432FA350132
:105DBA0064360164370150380A643C00643E003C92
:105DCA003F000040FFFF411450420A5A430AC844A8
:105DDA0005324500B44600FA4701064802034C0062
:105DEA00FA4EFFFF500606510596520A32530B46E9
:105DFA00540A96560102570546580002590A465A4D
:105E0A0032FA5B010A5C0A325E000A5F00FE61FF39
:105E1A00FF64FFFF6600026701016A0A3C6B00002B
:105E2A006C32967300007400007801327901327E78
:105E3A00FFFF81FFFF84FFFF8500AF860001870017
:105E4A00FA89010A8A00009900009D0A969E0001BB
:105E5A009FFFFFFAFAFA000077010103020000032C
:105E6A0001FA0400FA0500030A0A5A0B001E0C0084
:105E7A00FA0D00030E00030F01641000961201329E
:105E8A00130AFA14020215000017010A1801FA1976
:105E9A0005321A010A1B01FA1C05321FFFFF20FFF7
:105EAA00FF23011E2400642A00FA2B00FA2C5078E2
:105EBA002D003C2E00462F001E30006432507834EC
:105ECA0032FA350164360164370150380A643C00FD
:105EDA00643E003C3F000040FFFF411450420A5A12
:105EEA00430AC84405324500B44600FA470103484C
:105EFA0002024C00FA4EFFFF500606510596520A5E
:105F0A0032530B46540A965601015705465800016A
:105F1A00590A465A32FA5B010A5C0A325E000A5F83
:105F2A0000FE61FFFF64FFFF6600026701016A0A63
:105F3A003C6B00006C3296730000740000780132EA
:105F4A007901327EFFFF81FFFF84FFFF85FFFF8615
:105F5A00FFFF87FFFF8901028A00009900009D0A5E
:105F6A00969E00019FFFFFFAFAFA0065006F00791A
:105F7A000083008D009700A100AC00B600C000CAE3
:105F8A0000D400DE00E800F2005B0063006A0072E1
:105F9A00007A008200890091009900A100A800B04F
:105FAA0000B800BF00C700CF00D600DF00E600EE51
:105FBA0000F600400046004C00520059005F0065A0
:105FCA00006B00710077007D00830089008F0095C7
:105FDA00009C00A200A800AE00B400BA00C000C62F
:0E5FEA0000CC00D200D900DF00E500EB00F192
:1035E70090004CE0D3940440149007BDE0FEA3E0A4
:1035F700FF905D4C126131E493F59980129007BDFD
:10360700E0FEA3E0FF905E60126131E493F59990CC
:1036170007BDE0FEA3E0FF905D4AE493FC740193CD
:10362700FDEFB50507EEB50403754D009007BD1214
:1036370061182275A71085F97285FA737E017F00DC
:10364700E57312610AE5722FFF50010E8E598F5AEA
:10365700900017E0FCA3E0FDEF2DFDEE3CFC8C5B3A
:103667008D5C2275A71085F97285FA737E017F003C
:10367700E57312610AE5722FFF50010E8E598F5ABA
:10368700AC2CAD2DEF2DFDEE3CFC8C5B8D5C22E56B
:103697005CF5FBE55BF5FCD29322E55CF5E9E55BC0
:1036A700F5EAD29422E55CF5EBE55BF5ECD29122E5
:1036B700E55CF5EDE55BF5EED29222E55CF5FDE51F
:1036C7005BF5FED28722E55CF5CEE55BF5CFD290C0
:1036D70022AE59AF5A74788E048F05FF1260FA8CA8
:1036E7005B8D5CAE59AF5A74788E048F05FF1261FB
:1036F700258C598D5AE55A455960137478C3955AE4
:10370700FFE49559FE8E598F5A785B12615EE57218
:10371700A85BB80015D3955C4010E572C3955CFFB4
:10372700E4955BFE8E5B8F5C8010E5722403C39586
:103737005CFFE4955BFE8E5B8F5C2290008DE0B4AE
:103747000104C2138002D21390008EE0B40104C2B8
:10375700148002D2149000CBE075F0DCA4FFAEF029
:10376700740A8E048F05FF1260FA9007B3ECF0A37A
:10377700EDF0A20D401674038C068D0712610A74D2
:10378700011200399007B1EEF0A3EFF07E017F0040
:10379700900089E012610A9000CCE08E048F05FF4B
:1037A7001260FA740AFF1260FA8D5F9000D5E07517
:1037B700F0DCA4FFAEF0740A8E048F05FF1260FAE6
:1037C7009007B7ECF0A3EDF09000D7E060139000FE
:1037D700D7E0F5F0741684FF7E00EF9007C1F08004
:1037E7000674649007C1F09000CDE0900071F090EE
:1037F7000117E090005BF09000A6E090005DF0906C
:1038070000CFE090005EF090007BE090005FF090CA
:103817000101E0900064F074E3900070F09000B64E
:10382700E0B40B0874E3900070F0805A9000B6E0A3
:10383700B419129000CCE0905F5F12008CE4939073
:103847000070F080419000B6E0B41E129000CCE00A
:10385700905F7D12008CE493900070F080289000B8
:10386700B6E0B428129000CCE0905FA712008CE479
:1038770093900070F0800F9000B6E0B44608900077
:10388700ADE0900070F0900074E0FE9000B3E0B5FA
:103897000633900076E0FE9000D1E0B50627900051
:1038A70075E0FE9000DFE0B5061B900078E0FE9023
:1038B7000086E0B5060F900077E0FE9000C1E06E4D
:1038C7007003023A7D90004CE0C3940550087402DF
:1038D700900102F0801C9000C1E064036006900034
:1038E700DFE060087407900102F08006740A900117
:1038F70002F0900086E0B4010674009000ECF090AE
:103907000086E0B4020674009000D1F0900086E0D3
:10391700B4030674009000DEF09000B3E060147406
:103927001890009AF074009006C7F074009006C8CB
:10393700F0800C740090009AF074189006C7F0900D
:1039470000D1E0D3940140147419900104F074007D
:103957009006CBF074009006CCF0800C74009001B8
:1039670004F074199006CBF09000C1E0B4030890FE
:1039770000DFE064026002800674009000DFF090D0
:1039870000DFE0B401089000C1E064036002801A20
:10399700741A900105F0740090009BF07400900673
:1039A700CFF074009006D0F080339000B3E0B402FB
:1039B7001A741A90009BF07400900105F07400903F
:1039C70006CFF074009006D0F08012740090009B30
:1039D700F07400900105F0741A9006CFF09000C1C2
:1039E700E0B402069000DFE06002801474049006E1
:1039F700DBF074059006DFF074069006E3F0802490
:103A070074009006DBF074009006DCF074009006FA
:103A1700DFF074009006E0F074009006E3F07400A5
:103A27009006E4F0D22C9000B3E0900074F0900080
:103A3700DFE0900075F09000D1E0900076F0900004
:103A4700C1E0900077F0900086E0900078F0900059
:103A570086E090005CF09000C1E0900060F090007C
:103A6700DFE0900061F09000B3E0900062F090001A
:103A7700D1E0900063F09000E9E0B40117900023D3
:103A8700740FF0A374FFF0900025E4F0A3F0740224
:103A97009000E9F09000E9E0B40341900025E0FED2
:103AA700A3E0FF900023E0FCA3E0FD126156741031
:103AB70012610A7408120039EF90006DF0EF70067A
:103AC70074FF90006DF074009000E9F0900024E01E
:103AD70090006EF0900023E090006FF090007AE085
:103AE70090003FF090003FE004900040F090003FCE
:103AF700E02402900041F0900040E0D39403400B93
:103B0700900040E0C39403900040F0900041E0D360
:103B17009403400B900041E0C39403900041F0757B
:103B270050019000C0E0900042F0900042E0D39432
:103B370003400F900042E0C39403900042F0D22666
:103B47008002C226900042E004900043F0900042B9
:103B5700E02402900044F0900043E0D39403400B2C
:103B6700900043E0C39403900043F0900044E0D3F7
:103B77009403400B900044E0C39403900044F02268
:103B8700C293C294C291C292C287C290E5B554EF64
:103B9700F5B5E5B554DFF5B5C296C295C2A0C29793
:103BA700C2A2C2A1E5B554BFF5B5E5B5547FF5B5D9
:103BB700E5B554FBF5B5C215755D469000C3E070D9
:103BC70005756C028003756C03755400755300907E
:103BD700000C74FFF0A374DCF0C21BC21DC21F747B
:103BE700C8900039F074C890003BF074C890003D4D
:103BF700F0755200755100C20D754600E56EB409A7
:103C070003756E00756200900019E4F0A3F0756FFC
:103C170010C218C219C21A9007B3E0FEA3E0FF74DE
:103C27000312610A74011200399007B1EEF0A3EF95
:103C3700F0C202755600755500900010E4F0A3F02D
:103C4700C22D755800755700900085E075F032A4B5
:103C5700FDACF0900021ECF0A3EDF0900037747507
:103C6700F0A37430F0C20EC20FC23D2275A71085B3
:103C7700F97285FA737E017F00E57312610AE572B6
:103C87002FFF50010E8E598F5AAC5BAD5CEF2DFDA7
:103C9700EE3CFC8C5B8D5C1236961236A11236AC6C
:103CA7009000C1E0B403091236B71236C21236CDFE
:103CB70075A7002285F97285FA737E017F00E57387
:103CC70012610AE5722FFF50010E8E598F5A7E013D
:103CD7007F769000FEE012610AAC59AD5AED2FFFD6
:103CE700EC3EFE8E5B8F5CE55CF5EDE55BF5EE90FB
:103CF7000071E4F07412900048F02285F97285FA99
:103D0700737E017F00E57312610AE5722FFF500190
:103D17000E8E598F5A9007B3E0FCA3E0FDEF2DFDFF
:103D2700EE3CFC8C5B8D5CE55CF5FDE55BF5FE220E
:103D3700056322A2DBB340089000CDE0900071F04C
:103D4700A2DCB34006C296C295C2A075D8402285B0
:103D5700A77175A7109000C1E0640360079000DFAA
:103D6700E0B4022CA2D8B34002C293A2D9B3400256
:103D7700C294A2DAB34002C291A2DBB34002C2925C
:103D8700A2DCB34002C287A2DDB34002C290802DFD
:103D9700A2D8B3400AC2939000DFE06002C292A2A9
:103DA700D9B3400AC2949000DFE06002C287A2DA6A
:103DB700B3400AC2919000DFE06002C29075D8401C
:103DC7008571A722900047E4936406600280FE7421
:103DD700C89007B9F8E4F0E8A3F075B50075840159
:103DE70075A70075FFA0900045E4F075C91075A789
:103DF7000F75A1C775A70075D90075CE0C75A70FEC
:103E070075F1FE75F2FF75F30775F47875A4BA7549
:103E1700A5FF75A60775AE0075AFFF75D48175D57B
:103E2700FF75D6FF75D7FF75A70075A20175A14766
:103E370075F80975D80075D90475DD0975DE09753A
:103E4700D84075A71075D80075D90475DA0975DBE0
:103E57000975DC0975DD0975DE0975DF0975D84057
:103E670075A70075E60875E71075BC0175BE047582
:103E7700BD6C75BE0775BDA075BE0875BD0175BC67
:103E87000075BB1875BC2075BA0875E88075D11325
:103E970075A70F75E10575E20075C740123B877579
:103EA7009700759780740A1260EA7597C0E5975472
:103EB70020700280F8758F0275A700D2AF75980041
:103EC70075A90C75A70F75AB4375ADFB75AC1E7562
:103ED700A71075C91875CA0075CB0075C80475A7F2
:103EE70000758912758E04758C00758A00C2A9D277
:103EF7008C758D00758B00D2ABD28E75EF0675D998
:103F070044C29974C8F5097508001200E375B50035
:103F17001204E374639007B9F8E4F0E8A3F012031E
:103F27006F74C89007B9F8E4F0E8A3F07464F50972
:103F37007508001200E390005CE0900086F0C22351
:103F4700900086E0D3940340067400900086F090BA
:103F57000086E090595FF82828738028A2B44002B1
:103F6700D223802075A70F75F30F75A700A2A34072
:103F770002D223800F75A70F75F31775A700A2A4A8
:043F87004002D223FF
:0C595F00023F61023F63023F6B023F7C8D
:103F8B00A223B34066757208E572D3940E5020E5F8
:103F9B00729007B9F8E4F0E8A3F012023E7464F5EE
:103FAB00097508001200E37872740126F650D97473
:103FBB00029000C2F0900086E0D394034006740098
:103FCB00900086F0900086E090596BF8282873805B
:103FDB001674009000ECF0800E74009000D1F0800D
:073FEB000674009000DEF0F7
:0C596B00023FDA023FDC023FE4023FECA6
:103FF200D2228064757201E572D394075020E57273
:104002009007B9F8E4F0E8A3F012023E7464F509EF
:104012007508001200E37872740126F650D9740113
:104022009000C2F0900086E0D394034006740090A2
:104032000086F0900086E0905977F8282873801661
:1040420074009000ECF0800E74009000D1F08006B5
:0640520074009000DEF096
:0C59770002404002404202404A024052FE
:10405800C22290005BE0900117F090005CE09000B5
:1040680086F090005DE09000A6F090005EE0900081
:10407800CFF090005FE090007BF0900060E090004F
:10408800C1F0900061E09000DFF0900062E09000E5
:10409800B3F0900063E09000D1F0900064E09001EC
:1040A80001F09000CCE07006740A9000CCF090000B
:1040B800ADE0700674E39000ADF09000B3E00490BA
:1040C8000074F0123742E5B54401F5B57406900066
:1040D8004AF0740190004BF0740390004DF07405A1
:1040E80090004EF0742890004FF07405900050F046
:1040F80090004CE0B404067404900050F0740090F2
:104108000051F07400900056F07400900057F0745D
:1041180001900058F07400900059F074FF90005A14
:10412800F0744E900150F07469900151F0747390DE
:104138000152F07473900153F07461900154F0745B
:104148006E900155F07420900156F0743690015726
:10415800F07443900158F07479900159F0746C90A0
:10416800015AF0742090015BF0742090015CF074A7
:104178002090015DF0742090015EF09000E8E090DE
:10418800006DF090009FE090006EF09000A0E0902D
:10419800006FF0A2B6B39211A2B3B39212A2A4B365
:1041A8009229A2B4B3922AA2A3B3922B900069E4F5
:1041B800F0756E00743A900779F074FD90077AF004
:1041C80090006AE4F09007B3E0FEA3E0FF740312E6
:1041D800610A74011200399007B1EEF0A3EFF0758F
:1041E8006D01900048E4F0C228756200C216D2172B
:1041F800C202757000C22FD203C230D204C231D2BB
:1042080005C232D206C233D207C234D208C235D26E
:1042180009C236D20AC237D20BC238D20CC224C263
:1042280025C226C227C22C12009E755E00756A0040
:104238007560007564327565007566007567007590
:104248006800756900900019E4F0A3F0756B00D25E
:10425800B2D2A4D2B0D2B1D2A3D2A7D2A6D2A5D27A
:10426800B7900085E0D394FA400674FA900085F080
:104278007E017F0090006FE012610A90006EE02FCF
:10428800FF50010E900023EEF0A3EFF0EFD394FF60
:10429800EE940F4007900023E4F0A3F090006DE047
:1042A800700674FF90006DF074009000ACF0900000
:1042B800C2E0D39402400674019000C2F09000C39B
:1042C800E07005756C028003756C039000C4E0D340
:1042D8009401400674009000C4F09000CAE0C394B2
:1042E8000A5006740A9000CAF09000D4E070067470
:1042F800019000D4F09000D4E0B4FF0674FE900062
:10430800D4F09000DBE0D394FE400674FE9000DB0E
:10431800F0900101E0D3940240067401900101F08D
:10432800900117E0D3940140067401900117F074CE
:10433800019000E1F074019000E2F074009000E94F
:10434800F07400900109F074299006BFF0742A9067
:1043580006C3F0741B9006D3F0741C9006D7F0D2F5
:104368009C9000B4E0D39404400674049000B4F028
:104378009000E6E0D39404400674049000E6F0E56B
:104388006FD394104003756F109006C0E0D3940C5F
:10439800400674009006C0F09006C4E0D3940C4028
:1043A8000674009006C4F09006C8E0D3940C40064A
:1043B80074009006C8F09006CCE0D3940C400674C4
:1043C800009006CCF09006D0E0D3940C4006740020
:1043D8009006D0F09006D4E0D3940C400674009078
:1043E80006D4F09006D8E0D3940C400674009006EA
:1043F800D8F09006DCE0D3940C400674009006DCFC
:10440800F09006E0E0D3940C400674009006E0F0CB
:104418009006E4E0D3940C400674009006E4F0D2D1
:10442800EC75CF01A298B34005C298120616E54D67
:104438006006A299B3B340028005C299120AB4E596
:104448004E64016005E54EB4040280D5C28E7E102C
:104458007F00E56312610AE58D75F010A4FDACF0EC
:10446800EF2DFDEE3CFCE58B75F01084FF7E00ED32
:104478002FFFEC3EFE8E538F54D28E9000A6E06044
:104488005690001B12611890001BE0FCA3E0FD9001
:10449800001DE0FAA3E0FBEDB5033CECB50238B231
:1044A80021A20DB34013A221B34008E5B54404F599
:1044B800B58006E5B554FBF5B590001DE0FEA3E018
:1044C800FF90001FE0FCA3E0FDEF2DFDEE3CFC900B
:1044D800001DECF0A3EDF09000B3E060099000B38C
:1044E800E0C394034002806F1229C0A20DB35009A3
:1044F800900069E0C3940B4002800690009DE0F5AF
:1045080045E54575F005A4FFAEF09007BBEEF0A3B6
:10451800EFF090008AE0C395604007E55EC3955FC1
:1045280050079007BBE4F0A3F0AE2EAF2F9007BB67
:10453800E0FCA3E0FDEFD39DEE9C4004C297800B06
:10454800900069E0C394115002D2979000B3E0B490
:104558000205A297B392A19000B3E0B4031C122AFB
:10456800DBAE2EAF2F9007BBE0FCA3E0FDEFD39DA1
:10457800EE9C4004D2978002C297A2B6301101B3D4
:104588005003024ADDA2B6301101B35003024ADDDE
:10459800A2B6301301B3500302490D756D00055DD5
:1045A800A20EB35003024661E56CB4032EA22DB3EC
:1045B8004022E55DB40703756C01E55DC3940750BF
:1045C800069000487401F0E55DD394074006740234
:1045D800900048F0755D01D22D805AE56CB4020652
:1045E800756C01755D04E55DB40405755D01804574
:1045F800900048E07030E55DC39404500690004890
:104608007401F0E55DD3940440067402900048F00C
:10461800E55DC394045002D228E55DD394044002BA
:10462800D228C296C2959000C3E0B40105123B8718
:104638008003755D01C20EC20FA2269225A2B4B3F3
:104648004002C22AA2A4B34002C229A2A3B34002D4
:10465800C22BA228B34002C228E56CC394035006BB
:10466800E55D640460028016B225755D01A20F4005
:1046780004B20F80097405900048F0123B8790003F
:10468800C1E0B40308900042E0655D6002800BA2BF
:1046980025B34004D2278002C227E55DB4034990C0
:1046A80000A6E0604390001BE0FEA3E0FF9000A698
:1046B800E08E048F05FF1260FA74018C068D0712D4
:1046C800003990001FEEF0A3EFF090001FE0F8A370
:1046D800E090001DC8F0A3C8F090001BE4F0A3F020
:1046E800C221E5B554FBF5B5AE57AF58AC53AD5440
:1046F800EF2DFDEE3CFC8C578D58AE53AF54EFD3E5
:104708009DEE9C4011900013E0FAA3E0FBEBC394EC
:10471800E8EA9403400280069000131261189000A2
:104728000CE553F0A3E554F090000EE553F0A3E533
:1047380054F0AE53AF54740C8E048F05FF1260FA18
:104748008C558D56C28E758D00758B0075630075FE
:104758005401755300D28E90000CE0FEA3E0FFEFE9
:104768004E600B7CAC7D60125FF88E518F52AE515B
:10477800AF527428BE00039F5010E5622FFF50010E
:104788000E74011200398E518F528552629000CA00
:10479800E0A851B8000DD395524008E55290004763
:1047A800F080099000CAE014900047F0E56C6006BC
:1047B800755200755100E55D64016005E55DB4035F
:1047C800099000B3E0600312202BE56EB40903756D
:1047D8006E00A216500302488690007FE0B4017371
:1047E800900101E0B40214120C55900072E075F0CB
:1047F800BEA4FFAEF08E5B8F5C8056E56675F00A4E
:1048080084FF7E00900579126131E0F55A755900F0
:10481800AE59AF5A9000A4E012610A74648E048FF6
:1048280005FF1260FA8C5B8D5CE55C900012F0AEBF
:1048380059AF5A90007DE012610A74648E048F05A6
:10484800FF1260FA74BE8C068D0712610A8E5B8FA8
:104858005C801790007DE075F0BEA4FFAEF08E5B23
:104868008F5C9000A4E0900012F0E560C394CC50F7
:104878000690007DE070028003123C73D216E56C4E
:10488800B40106A215B3B340028009756F01900008
:10489800497401F0E56C70689000C6E0600D900006
:1048A80071E0A851B800069552400280299000C6D0
:1048B800E0B40208756F03756B00800CC200756B5D
:1048C80000900019E4F0A3F0900071E0600674090C
:1048D800900048F0802A756F0190003FE0B55D06B2
:1048E8009000497401F0900040E0B55D06740290B4
:1048F8000049F0900041E0B55D067403900049F06E
:10490800A213B39211A213B330B601B35003024AF3
:10491800DD756D01E5B54401F5B5740B900069F0DE
:10492800A2139211E55DD394484014D215E55DD3E6
:10493800944E400B7405900048F0D228755D46905F
:1049480000CEE0B40107E569C3941440028009125F
:104958003B877413900048F0A215B3B35018900029
:1049680037E0FEA3E0FF740212610AAC53AD54EFC6
:10497800C39DEE9C40028002D20E900037E553F0B2
:10498800A3E554F0A22F300301B35017A22FB34070
:1049980008E5B54408F5B58006E5B554F7F5B5A2C0
:1049A8002F9203A230300401B35017A230B340084D
:1049B800E5B54402F5B58006E5B554FDF5B5A23078
:1049C8009204A231300501B3500FA231B34004D292
:1049D800978002C297A2319205A232300601B350E5
:1049E8000FA232B34004D2A28002C2A2A23292061F
:1049F800A233300701B3500FA233B34004D2A180D1
:104A080002C2A1A2339207A234300801B35017A200
:104A180034B34008E5B54440F5B58006E5B554BF64
:104A2800F5B5A2349208A235300901B35017A23562
:104A3800B34008E5B54480F5B58006E5B5547FF583
:104A4800B5A2359209A236300A01B3500FA236B387
:104A58004004D2928002C292A236920AA237300B48
:104A680001B3500FA237B34004D2878002C287A295
:104A780037920BA238300C01B3500FA238B3400460
:104A8800D2908002C290A238920CE569C39441503A
:104A980009740E900048F0123B87900050E0FE9099
:104AA800004CE004C39E400990004CE0D3940640BB
:104AB8000974FB900048F0123B87900055E06015A0
:104AC800900055E0FE90004FE06E600974FE900083
:104AD80048F0123B87A228B34006C296C295C2A0EE
:104AE8009000FEE0600CAE51AF527414BE00059FFA
:104AF80040028048900086E0905983F82828738007
:104B08003BA2B4B35005A22AB340028005123CBBB5
:104B1800D22A8028A2A3B35005A22BB34002800555
:104B2800123CBBD22B8015A2A4B35005A229B340D6
:0C4B3800028005123CBBD22980028000E4
:10598300024B07024B09024B1C024B2F024B4202F4
:025993004B4483
:104B4400A218B3B35008900042E0655D6003024BC5
:104B5400D9A201B35006A200B3B340028071900001
:104B6400C1E0B4034312363AA20DB34021A227B3E5
:104B7400400512369680031236B79000DFE0B40188
:104B84000BA202B34004D2A18002C2A18018123643
:104B9400961236B79000DFE0B4010BA202B34004D2
:104BA400D2A18002C2A180249000DFE0C39402500D
:104BB4000F12363A123696A202B34002D292800CF9
:104BC40012363A12369612366A1236B775A700C2F2
:104BD40018D219D21AA219B3B35008900043E06551
:104BE4005D6003024C6EA201B35006A200B3B34051
:104BF4000280719000C1E0B4034312363AA20DB3AF
:104C04004021A227B340051236A180031236C29078
:104C140000DFE0B4010BA202B34004D2A18002C2BF
:104C2400A180181236A11236C29000DFE0B4010B45
:104C3400A202B34004D2A18002C2A180249000DF6A
:104C4400E0C39402500F12363A1236A1A202B340C6
:104C540002D287800C12363A1236A112366A123604
:104C6400C275A700D218C219D21AA21AB3B3500837
:104C7400900044E0655D6003024D03A201B3500659
:104C8400A200B3B3400280719000C1E0B4034312A8
:104C9400363AA20DB34021A227B340051236AC80A8
:104CA400031236CD9000DFE0B4010BA202B340043E
:104CB400D2A18002C2A180181236AC1236CD900067
:104CC400DFE0B4010BA202B34004D2A18002C2A16E
:104CD40080249000DFE0C39402500F12363A12365B
:104CE400ACA202B34002D290800C12363A1236AC17
:104CF40012366A1236CD75A700D218D219C21AE537
:0F4D04006F905995F828287302513E9000E6E011
:06599500024D0C024D0F53
:104D13009059C8F8282873121B078012121B0780AA
:0E4D23000D121B918008121C3D8003121C3DD6
:0F59C800024D1A024D1F024D24024D29024D2E91
:104D3100756F0202513E121D69121E80A23DB340E1
:104D41000C9000A8E0F56B7410900048F090007989
:104D5100E0256BF5349007B1E0FEA3E0FF74141277
:104D6100610A90000EE0FCA3E0FD74068F02FF12C1
:104D710060FA8D078C038E048A058B06125FF8900A
:104D810007B5EEF0A3EFF09000CFE0B40108744650
:104D9100BE00059F4002800D74469007B5F8E4F00F
:104DA100E8A3F0801B9007B5E0FEA3E0FF74F0BE1E
:104DB10000039F500B74F09007B5F8E4F0E8A3F0FE
:104DC100E53470037534019007B5E0FEA3E0FFE51B
:104DD100342FFF50010E9007B5EEF0A3EFF0756F81
:054DE10003900049E011
:03599B00024D3783
:104DE6009059D7F82828738019A23E4003756F0A98
:104DF6008010A23E4003756F0B8007A23E400375EC
:024E06006F0C2F
:0C59D700024DED024DEF024DF8024E01B2
:104E080002513E9006C0E060031221149000FFE0BA
:104E1800B40114900100E0A851B80004955250075D
:104E2800E55EC3955F40028003024EB59000B4E092
:104E3800D39402403F900088E02403A851B80004AE
:104E48009552500990008AE0D3956050028008D2AC
:104E5800017408900048F0900088E0A851B8000557
:104E6800D39552500B90008AE02403C395605002FA
:104E7800C2018039900088E02403A851B800049545
:104E8800525007E55EC3955F40028008D20174085E
:104E9800900048F0900088E0A851B80005D39552DA
:104EA8005009E55F240FC3955E5002C2019000CE01
:104EB800E07007E569C3941440028002D201A201A0
:104EC8004005756F04800A756F10900019E4F0A30F
:104ED800F0A20DB34029E56675F00A84FF7E0090C4
:104EE8000579126131E0C394695005122060800F82
:104EF8009007B3E0F8A3E09007B1C8F0A3C8F002A8
:064F0800513E9000B4E0F0
:06599E00024E0B024F0A4D
:104F0E009059E3F8282873120D3F8012120D3F803E
:0E4F1E000D120EED8008120F9F8003120F9FE0
:0F59E300024F15024F1A024F1F024F24024F2985
:104F2C009006C4E060031221F0756F0502513E1229
:104F3C0010AB756F069006C8E060031222E0900675
:104F4C00CCE060031223BC02513E900012E06006DC
:104F5C00A20DB3B34002801D900012E02529FFAED4
:104F6C002850010E8E288F29E55DD39401500690B0
:104F7C000012E014F01212F1756F079006D0E06089
:104F8C00031224989006D4E0600312257402513E5B
:104F9C00900101E0B40203120CCD12154E756F088E
:104FAC009006D8E060031226509006DCE0600312F5
:104FBC00272C02513E12190AA218B35005A219B39C
:104FCC0040028006D218D219D21A756F109006E0E2
:104FDC00E060031228089006E4E060031228E40263
:104FEC00513E02513E90003AE0C394465008C2969E
:104FFC00744690003AF085345A75590090003FE0A1
:10500C00F5721236D8E55C90003AF0900006E5593E
:10501C00F0A3E55AF0C21C9007B5E0F559A3E0F5F2
:10502C005A90003FE0F5721236D8E55C900039F0EA
:10503C00900000E559F0A3E55AF0C21BE56CB401F1
:10504C0005756F0B8003756F0302513E90003CE0B9
:10505C00C3944650139000CFE0B40104C296800272
:10506C00C295744690003CF085345A7559009000F6
:10507C0040E0F5721236D8E55C90003CF0900008E8
:10508C00E559F0A3E55AF0C21E9007B5E0F559A317
:10509C00E0F55A900040E0F5721236D8E55C9000CD
:1050AC003BF0900002E559F0A3E55AF0C21DE56C07
:1050BC00B40105756F0C8003756F03807590003E0D
:1050CC00E0C3944650139000CFE0B40104C2968024
:1050DC0002C2A0744690003EF085345A7559009077
:1050EC000041E0F5721236D8E55C90003EF090007D
:1050FC000AE559F0A3E55AF0C2209007B5E0F5593E
:10510C00A3E0F55A900041E0F5721236D8E55C90B8
:10511C00003DF0900004E559F0A3E55AF0C21FE5FC
:10512C006CB40103756C00756F03800680048002FB
:02513C008000F1
:1059A400024F3B024F56024F9C024FC1024FEE0280
:1059B4004FF10250580250C902513802513A025173
:0459C4003C02513E12
:10513E00900039E0B55D0280030251D9A21B406B8D
:10514E00900000E0FEA3E0FFEF4E605DAC51AD526B
:10515E00740ABC0033D39D402FAA55AB5674058AF2
:10516E00048B05FF1260FA8D068C07900000E0FCA0
:10517E00A3E0FDCFCECF12000374011200399000D0
:10518E0000EEF0A3EFF08021AE55AF56900000E098
:10519E00FCA3E0FD120003740A8E048F05FF12605B
:1051AE00FA900000ECF0A3EDF0D21BAE53AF54908A
:1051BE000000E0FCA3E0FDEFC39DEE9C400D123D10
:1051CE0002D296C21B74C8900039F0A21BB3B35022
:1051DE0007900039E0B55D02800D123D02D2967443
:1051EE00C8900039F0C21B90003AE0B55D02800312
:1051FE0002528DA21C406B900006E0FEA3E0FFEF72
:10520E004E605DAC51AD52740ABC0033D39D402F3D
:10521E00AA55AB5674058A048B05FF1260FA8D06EB
:10522E008C07900006E0FCA3E0FDCFCECF1200036A
:10523E007401120039900006EEF0A3EFF08021AE5B
:10524E0055AF56900006E0FCA3E0FD120003740A71
:10525E008E048F05FF1260FA900006ECF0A3EDF0BD
:10526E00D21CAE53AF54900006E0FCA3E0FDEFC39A
:10527E009DEE9C400AC296744690003AF0C21CA263
:10528E001CB3B3500790003AE0B55D02800AC29697
:10529E00744690003AF0C21C90003BE0B55D02806F
:1052AE000302534CA21D406B900002E0FEA3E0FFF0
:1052BE00EF4E605DAC51AD52740ABC0033D39D40CD
:1052CE002FAA55AB5674058A048B05FF1260FA8D12
:1052DE00068C07900002E0FCA3E0FDCFCECF1200BB
:1052EE00037401120039900002EEF0A3EFF080215A
:1052FE00AE55AF56900002E0FCA3E0FD1200037421
:10530E000A8E048F05FF1260FA900002ECF0A3EDF6
:10531E00F0D21DAE53AF54900002E0FCA3E0FDEFBF
:10532E00C39DEE9C4018123D029000CFE0B40104E4
:10533E00D2968002D295C21D74C890003BF0A21D79
:10534E00B3B3500790003BE0B55D028018123D02EA
:10535E009000CFE0B40104D2968002D29574C8902A
:10536E00003BF0C21D90003CE0B55D02800302548C
:10537E0016A21E406B900008E0FEA3E0FFEF4E6009
:10538E005DAC51AD52740ABC0033D39D402FAA556B
:10539E00AB5674058A048B05FF1260FA8D068C07D6
:1053AE00900008E0FCA3E0FDCFCECF120003740105
:1053BE00120039900008EEF0A3EFF08021AE55AF49
:1053CE0056900008E0FCA3E0FD120003740A8E0460
:1053DE008F05FF1260FA900008ECF0A3EDF0D21EDC
:1053EE00AE53AF54900008E0FCA3E0FDEFC39DEE7A
:1053FE009C40159000CFE0B40104C2968002C29585
:10540E00744690003CF0C21EA21EB3B3500790002B
:10541E003CE0B55D0280159000CFE0B40104C29669
:10542E008002C295744690003CF0C21E90003DE092
:10543E00B55D0280030254E0A21F406B900004E0B1
:10544E00FEA3E0FFEF4E605DAC51AD52740ABC009E
:10545E0033D39D402FAA55AB5674058A048B05FF96
:10546E001260FA8D068C07900004E0FCA3E0FDCFDD
:10547E00CECF1200037401120039900004EEF0A397
:10548E00EFF08021AE55AF56900004E0FCA3E0FD96
:10549E00120003740A8E048F05FF1260FA90000446
:1054AE00ECF0A3EDF0D21FAE53AF54900004E0FC2D
:1054BE00A3E0FDEFC39DEE9C4018123D029000CF7D
:1054CE00E0B40104D2968002D2A0C21F74C890002C
:1054DE003DF0A21FB3B3500790003DE0B55D0280D2
:1054EE0018123D029000CFE0B40104D2968002D291
:1054FE00A074C890003DF0C21F90003EE0B55D0262
:10550E0080030255AAA220406B90000AE0FEA3E0A1
:10551E00FFEF4E605DAC51AD52740ABC0033D39DAB
:10552E00402FAA55AB5674058A048B05FF1260FAFC
:10553E008D068C0790000AE0FCA3E0FDCFCECF12C3
:10554E000003740112003990000AEEF0A3EFF08010
:10555E0021AE55AF5690000AE0FCA3E0FD12000309
:10556E00740A8E048F05FF1260FA90000AECF0A305
:10557E00EDF0D220AE53AF5490000AE0FCA3E0FD54
:10558E00EFC39DEE9C40159000CFE0B40104C2968F
:10559E008002C2A0744690003EF0C220A220B3B397
:1055AE00500790003EE0B55D0280159000CFE0B44C
:1055BE000104C2968002C2A0744690003EF0C22042
:1055CE009000D1E0B4020280030256EA90006BE034
:1055DE00D39565506490006BE0F4042565FE900051
:1055EE00D4E08E00F5F0E884FF7E008F72EFC39456
:1055FE0010500CEF8572F0A4FDACF08D7280037527
:10560E0072FF90006BE0D39572400B90006BE0C37D
:10561E009572F57080037570009000EFE0D3957071
:10562E0040069000EFE0F5709000F0E0C3957050EA
:10563E00069000F0E0F570807190006BE0C3956508
:10564E00FE9000D4E08E00F5F0E884FF7E008F72AD
:10565E00EFC39410500CEF8572F0A4FDACF08D7278
:10566E0080037572FF85725A75590090006BE025A4
:10567E005AFFAE5950010E8E598F5A74FFBE000953
:10568E00D39F4005855A7080037570FF9000EFE040
:10569E00D3957040069000EFE0F5709000F0E0C3F7
:1056AE00957050069000F0E0F570A20DB3B3500D5A
:1056BE0090006CE0FE9000DCE0D39E5002800A74F5
:1056CE0007900048F0C2A2801375A710E5CDC395D0
:1056DE00704004C2A28002D2A275A700E56EC394E8
:1056EE0009500AA2EDB34005C2ED122C7AAE53AFAB
:1056FE00547450C39F74C39E400C90006AE0C394D0
:10570E005A400302595CA215B34009123B87740636
:10571E00900048F0A223B34008E5B54404F5B580E7
:10572E0006E5B554FBF5B5A217B3500EE560D3945C
:10573E00334007E560C394CC4002802FE5B54401A9
:10574E00F5B5740B900069F090007DE075F0BEA485
:10575E00FFAEF08E5B8F5C7402BE000AD39F4006D4
:10576E00755C02755B00123C73D21790006AE0D331
:10577E0094014007E560C3941A40028002C217905C
:10578E0006C0E06003122114A22F300301B350179C
:10579E00A22FB34008E5B54408F5B58006E5B5542B
:1057AE00F7F5B5A22F92039006C4E060031221F024
:1057BE00A230300401B35017A230B34008E5B5440F
:1057CE0002F5B58006E5B554FDF5B5A2309204900C
:1057DE0006C8E060031222E0A231300501B3500F7B
:1057EE00A231B34004D2978002C297A231920590A3
:1057FE0006CCE060031223BCA232300601B3500F78
:10580E00A232B34004D2A28002C2A2A23292069069
:10581E0006D0E06003122498A233300701B3500F74
:10582E00A233B34004D2A18002C2A1A23392079048
:10583E0006D4E06003122574A234300801B3501769
:10584E00A234B34008E5B54440F5B58006E5B5543D
:10585E00BFF5B5A23492089006D8E0600312265028
:10586E00A235300901B35017A235B34008E5B5444F
:10587E0080F5B58006E5B5547FF5B5A23592099051
:10588E0006DCE0600312272CA236300A01B3500F5B
:10589E00A236B34004D2928002C292A236920A90ED
:1058AE0006E0E06003122808A237300B01B3500F58
:1058BE00A237B34004D2878002C287A237920B90E0
:1058CE0006E4E060031228E4A238300C01B3500F56
:1058DE00A238B34004D2908002C290A238920C90AB
:1058EE00006AE0C3945A5010E56EB4090990006A3C
:1058FE00E004F0756E00803BE56EB40903756E0032
:10590E00755400755300758D00758B00756300908E
:10591E000069E0C394115008900069E004F080061D
:10592E007411900069F0900069E0B41106E5B55469
:10593E00FEF5B590006AE0D394014007E569C39483
:10594E004140028009740E900048F0123B870244D9
:01595E00291F
:1059F2000000010001400160018001A001C001E03E
:105A020002000300039603B603D603F40400050064
:105A12000512052405360548055A056C057E0590D4
:105A220005A805C005DE0600061406280646066E11
:105A320006AE00FF013F015F017F019F01BF01DF51
:105A420001FF02FF039503B503D503F303FF04FF30
:105A520005110523053505470559056B057D058F9C
:105A620005A705BF05DD05F1061306270645066DE8
:105A720006AD06ED0FAA0FA50F9F0F9A0F940F8D7B
:105A82000F870F800F780F710F680F600F570F4E3F
:105A92000F450F3B0F300F250F1A0F0E0F020EF599
:105AA2000EE80EDB0ECC0EBE0EAE0E9F0E8E0E7DDF
:105AB2000E6C0E5A0E470E340E200E0C0DF70DE230
:105AC2000DCB0DB50D9D0D850D6D0D540D3A0D20AF
:105AD2000D050CE90CCE0CB10C940C760C580C3A5A
:105AE2000C1B0BFB0BDB0BBB0B9A0B790B570B3510
:105AF2000B130AF10ACE0AAB0A870A640A400A1C8F
:105B020009F809D409B0098C09670943091F08FB80
:105B120008D608B2088E086A0846082307FF07DC81
:105B220007B9079607730751072F070D06EC06CA38
:105B320006AA068906690649062A060A05EC05CD63
:105B420005B0059205750558053C0520050504EAD2
:105B520004CF04B5049C048204690451043904226C
:105B6200040B03F403DE03C803B2039D0389037528
:105B72000361034D033B03280316030402F202E10F
:105B820002D102C002B002A0029102820273026537
:105B920002570249023C022F02220216020901FDAB
:105BA20001F201E601DB01D001C601BB01B101A78F
:105BB200019D0194018B01820179017001680160EC
:105BC200015801500148014101390132012B0125DF
:105BD200011E01180111010B010500FF00FA0FA6B9
:105BE2000FA00F990F920F8B0F840F7C0F740F6B06
:105BF2000F620F580F4E0F430F380F2C0F1F0F124B
:105C02000F050EF70EE80ED80EC80EB70EA50E93AE
:105C12000E800E6C0E580E420E2C0E150DFD0DE46C
:105C22000DCB0DB10D950D790D5D0D3F0D200D01C3
:105C32000CE10CC00C9E0C7C0C590C350C100BEAC0
:105C42000BC40B9E0B760B4F0B260AFD0AD40AAA35
:105C52000A800A550A2A09FF09D409A8097C0950B1
:105C6200092508F908CD08A10875084A081E07F396
:105C720007C8079D07730749072006F706CE06A641
:105C8200067E06570630060A05E405BF059B057722
:105C920005540532051004EF04CE04AE048F0471DE
:105CA20004530435041903FD03E203C703AD03944F
:105CB200037B0363034B0334031E030802F302DE78
:105CC20002CA02B602A30291027F026D025C024C7A
:105CD200023C022C021D020E020001F201E401D775
:105CE20001CA01BE01B101A6019A018F0185017AA3
:105CF20001700166015D0153014A0141013901311F
:105D02000129012101190112010B010400FD00F713
:105D120000F000EA00E400DE00D900D300CE00C9A2
:105D220000C400BF00BA00B500B100AD00A800A4D5
:105D320000A0009C009900950091008E008A0087C7
:085D420000840081007E007B5B
:10009E007547009007BDE4F0A3F075310075300090
:1000AE00754D00754E00C23AD23B74FE9007C7F8EC
:1000BE00E4F0E8A3F074FE9007C9F8E4F0E8A3F0CA
:1000CE00745A9007CBF0745A9007CCF0D23CC22EE3
:1000DE00C23EC23922750B00750A00AE0AAF0BACD8
:1000EE0008AD09EDC39FEC9E401674FF1260EA75D1
:1000FE00CF01780B740126F6500418E436F650DB67
:10010E0022900045E0B4AA1C900779E0B43C15900B
:10011E0007B9E0FEA3E0FFEF4E6009741EBE0004B7
:10012E00D39F500302023D755C00755B0075F809A4
:10013E009007B9E0FEA3E0FF74076F4E6006740EE1
:10014E006F4E7006743A900779F09007B9E0FEA3EF
:10015E00E0FF7408BE001ED39F401A7E017F0890F8
:10016E0007B9E0FCA3E0FD1DBDFF011C1200038ECC
:10017E00598F5A801F9007B9E0FEA3E0FF74081252
:10018E00614E8F048E057E017F08CDCCCD1200030B
:10019E008E598F5AAE5BAF5C740CD39F74019E5018
:1001AE0003020238A2F9B3407EE55C455B7003752D
:1001BE00A382AE5BAF5C74016F4E700375A300AE8D
:1001CE005BAF5C74026F4E700D9007BAE075F00273
:1001DE00A4FDACF08DA3AE5BAF5C74036F4E7003E9
:1001EE0075A300AE5BAF5C7403BE00039F5013ACEF
:1001FE0059AD5AED2FFFEC3EFE900075126131E0C5
:10020E00F5A3AE5BAF5CEFB40B09EEB4010574144D
:10021E001260EAAE5BAF5CEFB40B07EEB401037590
:10022E00F80D785B12615E0201A2900045E4F022A7
:10023E00755C00755B0075F8099007B9E0FEA3E0E8
:10024E00FF7408BE001ED39F401A7E017F089007E0
:10025E00B9E0FCA3E0FD1DBDFF011C1200038E5989
:10026E008F5A801F9007B9E0FEA3E0FF7408126159
:10027E004E8F048E057E017F08CDCCCD1200038EED
:10028E00598F5AAE5BAF5C7411D39F74019E5003AD
:10029E0002036EA2F9B3500302036BE55C455B707B
:1002AE000375A3D2AE5BAF5C74016F4E700375A382
:1002BE0000AE5BAF5C74026F4E700D9007BAE075C6
:1002CE00F002A4FDACF08DA3AE5BAF5C74036F4E79
:1002DE00700375A300AE5BAF5C74046F4E70037554
:1002EE00A300AE5BAF5C74056F4E700375A300AEDA
:1002FE005BAF5C74066F4E700375A300AE5BAF5CB4
:10030E0074076F4E700375A300AE5BAF5C74086F1D
:10031E004E700375A300AE5BAF5C7408BE00039F06
:10032E005016AC59AD5AED2FFFEC3EFE90007012F8
:10033E006131E5A3F075A300AE5BAF5CEFB41009BD
:10034E00EEB4010574141260EAAE5BAF5CEFB4104C
:10035E0007EEB4010375F80D785B12615E0202912F
:10036E0022755C00755B0075F809AE5BAF5C7417A7
:10037E00BE0004D39F5003020447A2F9B3500302F8
:10038E000444E55C455B700375A3D2AE5BAF5C7451
:10039E00016F4E700375A300AE5BAF5C74026F4EBF
:1003AE00700D9007BAE075F002A4FDACF08DA3AE0F
:1003BE005BAF5C74036F4E700375A300AE5BAF5CF6
:1003CE0074046F4E700375A300AE5BAF5C74056F63
:1003DE004E700375A300AE5BAF5C74066F4E700378
:1003EE0075A300AE5BAF5C74076F4E700375A30010
:1003FE00AE5BAF5C74086F4E700375A300AE5BAF5F
:10040E005C7408BE00039F500C900052126131E5DF
:10041E00A3F075A300AE5BAF5C74166F4E700574DF
:10042E00141260EAAE5BAF5C74166F4E700375F813
:10043E000D785B12615E02037822900045E0B4AB4A
:10044E000280030204E2755C00755B0075F809AE6C
:10045E005BAF5C7412BE007CD39F4078A2F9B340B0
:10046E0070E55C455B700375A382AE5BAF5C740197
:10047E006F4E700375A300AE5BAF5C74026F4E706F
:10048E000D9007BAE075F002A4FDACF08DA3AE5B43
:10049E00AF5C74036F4E700375A300AE5BAF5C74FC
:1004AE0003BE00039F5009900057126131E0F5A37F
:1004BE00AE5BAF5C74116F4E700574141260EAAED1
:1004CE005BAF5C74116F4E700375F80D785B126143
:1004DE005E02045D229007C4E4F074649007B9F8DC
:1004EE00E4F0E8A3F012036F74C89007B9F8E4F0D3
:1004FE00E8A3F090005EE0B4371A90005BE0900045
:10050E0052F090005CE0900053F090005DE090009F
:10051E0054F080469007C47401F074659007B9F8E2
:10052E00E4F0E8A3F012036F74C89007B9F8E4F092
:10053E00E8A3F090005EE0B4371A90005BE0900004
:10054E0052F090005CE0900053F090005DE090005F
:10055E0054F0800674029007C4F09007C5E4F0745E
:10056E00669007B9F8E4F0E8A3F012036F74C89030
:10057E0007B9F8E4F0E8A3F090005DE0B43712900C
:10058E00005BE090004CF090005CE0900055F08035
:10059E00769007C57401F074679007B9F8E4F0E837
:1005AE00A3F012036F74C89007B9F8E4F0E8A3F053
:1005BE0090005DE0B4371290005BE090004CF0903C
:1005CE00005CE0900055F0803E74029007C5F07418
:1005DE00689007B9F8E4F0E8A3F012036F74C890BE
:1005EE0007B9F8E4F0E8A3F090005DE0B43712909C
:1005FE00005BE090004CF090005CE0900055F080C5
:10060E000674039007C5F022E54E64046006E59972
:10061E0064FF6002802AA23A4004D23A8020E54E5E
:10062E00600874E6254E900048F0754E00E54D606A
:10063E000874F0254D900048F0754D00C23A8002C6
:10064E00C23AE54E9033F8F8282873754E00E599B6
:10065E00B4FF03754D01E599B4FE03754D02E5999E
:10066E00B4FD03754D03E599B4FC03754D04E5998E
:10067E00B4FA03754D05E599B4FB06754E01123BB0
:10068E0087E599B4F906754E04123B87E599D39424
:10069E00E54007E599C394F04002801685994F75A1
:1006AE004E027E017F00E54FC394E612610A8E3240
:1006BE008F339007BDE4F0A3F0E599D394C44007BF
:1006CE00E599C394E64002802885994F754E0374D0
:1006DE00E5C3954FF533753200AE32AF339059F214
:1006EE001260D9E493F87401939007BDC8F0A3C8C3
:1006FE00F0D299020AB390005BE070429007BDE021
:10070E00FEA3E0FF74FFBE00039F5009EFC39446A3
:10071E00EE940640119007BDE0FEA3E0FFEFD394E8
:10072E006DEE940640139007BDE0FEA3E0FF90002F
:10073E0079126131E599F0800385997380119007E4
:10074E00BDE0FEA3E0FF900079126131E599F090D3
:10075E0007BD1261189007BDE0FEA3E0FFEFB401E4
:10076E0006EEB40702800302089B900779E0B43CC2
:10077E00028003020885C29C90005BE0900117F096
:10078E0090005CE0900086F090005DE09000A6F096
:10079E0090005EE09000CFF090005FE090007BF064
:1007AE00900060E09000C1F0900061E09000DFF0FA
:1007BE00900062E09000B3F0900063E09000D1F002
:1007CE00900064E0900101F012374290006DE090CD
:1007DE0000E8F090006EE090009FF090006FE090C7
:1007EE0000A0F074639007B9F8E4F0E8A3F074ABDE
:1007FE00900045F0120448900045E4F075096475C8
:10080E0008001200E3A2224038757201E572D394FB
:10081E0007502CE5729007B9F8E4F0E8A3F074AA3B
:10082E00900045F012010FE572C394075009750947
:10083E00647508001200E37872740126F650CD80BC
:10084E0036757208E572D3940E502CE5729007B986
:10085E00F8E4F0E8A3F074AA900045F012010FE559
:10086E0072C3940E50097509647508001200E3787E
:10087E0072740126F650CD74C89007B9F8E4F0E80A
:10088E00A3F0D29C754E00754D007599FB020AB30C
:10089E009007BDE0FEA3E0FFEF4E7006859931751F
:1008AE0030009007BDE0FEA3E0FF74016F4E701B99
:1008BE00AC30AD31AA32AB33ED2BFBEC3AFA8A06F3
:1008CE008B07900079126131E599F09007BD1261A6
:1008DE00189007BDE0FEA3E0FF74026F4E7021ACCE
:1008EE0030AD3174566D4C7006E54F64E660028093
:1008FE0003123B87123742854F99754E00754D0096
:10090E00020AB39007BDE0FEA3E0FF9000791261EA
:10091E0031E599F09007BD1261189007BDE0FEA376
:10092E00E0FFAC32AD338F028E038C068D07905AEA
:10093E00341260D9E493F9740193FEEAD39EEB99D5
:10094E004009854F99754E00754D00020AB3900708
:10095E00BDE0FEA3E0FF900079126131E599F090C1
:10096E0007BD1261189007BDE0FEA3E0FFEFB400D3
:10097E0006EEB401028003020AB3900054E075F053
:10098E0002A4FDACF08D72ED90007912613CEDFA8F
:10099E00E0FBEA90007C12613CEBFAE0FBEA2BFAFA
:1009AE00900054E0B502028003020AA50DED9000FE
:1009BE007912613CE572FDE0FAED90007D12613C2A
:1009CE00EAFDE0FAEDC39AFD900054E0B505028011
:1009DE0003020AA5E57290007B12613CE572FDE010
:1009EE00FAED90007E12613CEAFDE0FAED2AFD90F0
:1009FE000054E0B505028003020AA5E57290007F5F
:100A0E0012613CFDE0FAED900054E0F4042A9000EF
:100A1E005BF0E57290008012613CFDE0FAED900013
:100A2E0054E0F4042A90005CF0E5729000811261AB
:100A3E003CFDE0FAED900054E0F4042A90005DF0E5
:100A4E00E57290008212613CFDE0FAED900054E0F8
:100A5E00F4042A9007B9F8E4F0E8A3F074AB900020
:100A6E0045F01204487509647508001200E39007FA
:100A7E00B91261181204487509647508001200E372
:100A8E009007B91261181204487599F975096475C1
:100A9E0008001200E380FE7599FF75096475080061
:050AAE001200E380FED0
:0F33F80002065902070402089E02091102095C2D
:100AB30022E54D903407F8282873020B989007BD60
:100AC300E0FEA3E0FF90004A126131E0F599900740
:100AD300BD1261189007BDE0FEA3E0FF74116F4ED5
:100AE3007003754D00020B98856D99020B98900762
:100AF300BDE0FEA3E0FF900079126131E0F599EFCC
:100B0300B40107EEB40703754D009007BD126118D9
:070B1300020B989007BEE001
:0F340700020ABD020AC0020AEB020AF1020B160A
:100B1A009035BAF82828738552998067855E99803E
:100B2A0062856099805D856499805885669980534D
:100B3A00856799804E85689980498569998044902E
:100B4A00001AE0F599803CA23BB340077599FAC2B6
:100B5A003B8017A22CB3400575990F800B90004873
:100B6A00E0F599900048E4F0C22C8017856A9980D4
:100B7A0012856599800D856B9980087599FC8003AB
:030B8A00754D00A6
:1035BA00020B21020B26020B2B020B30020B3502E7
:1035CA000B3A020B3F020B44020B49020B51020B4E
:0D35DA0076020B7B020B80020B85020B8A30
:0B0B8D009007BD12611880031235E7CD
:03341600020B9511
:100B980022E537255AFFAE5950010E9000791261AF
:100BA80031E0F538E537255AFFAE5950010E0FBF31
:100BB80000010E900079126131E0F539853F3BE57F
:100BC80038B539058538378041E539D39538401D22
:100BD800E539C39538853AF0A4FFAEF0E53B8E04BD
:100BE8008F05FF1260FAED2538F537801DE538C30B
:100BF8009539853AF0A4FFAEF0E53B8E048F05FFEA
:100C08001260FAEDF4042538F53722E539D3953822
:100C1800401DE539C39538853AF0A4FFAEF0E53BB1
:100C28008E048F05FF1260FAED2538F537801DE533
:100C380038C39539853AF0A4FFAEF0E53B8E048FB2
:100C480005FF1260FAEDF4042538F5372290007F8D
:100C5800E0B40170E56675F00A84FF7E008F37E521
:100C68006675F00A84ADF07C008D3A753F0A7559B7
:100C780005755A24E537C394115005120B9980065F
:100C88009005AEE0F537E537900072F0E56675F04F
:100C98000A84FF7E008F37E56675F00A84ADF07C24
:100CA800008D3A753F0A755905755A5AE537C39448
:100CB800115005120B9980069005E4E0F537E537E9
:100CC800900012F02290007FE0B4016AE56675F0AA
:100CD8000A84FF7E008F37E56675F00A84ADF07CE4
:100CE800008D3A753F0A755905755A36E537C3942C
:100CF800115005120B9980069005C0E0F53785372D
:100D08004BE56675F00A84FF7E008F37E56675F05F
:100D18000A84ADF07C008D3A753F0A755905755AFD
:100D280048E537C394115005120B9980069005D2F7
:100D3800E0F53785374C22E55E75F00484FF7E00C8
:100D48008F37E55E75F00484ADF07C008D3A753F11
:100D580004755901755A00E537C3943F5005120BC5
:100D68009980069001B8E0F53785372975280090F5
:100D78000047E075F020A4FFAEF09000CAE08E04B2
:100D88008F05FF1260FA8D379000B2E0D3955E5060
:100D980003020E459000D6E0D3955E4010ED900119
:100DA800B912613CE0F52B752A00020E429000A1B1
:100DB800E0D3955E4043E5379001B912613CE0F518
:100DC80038E5379001D912613CE0F5399000D6E05A
:100DD800F404255EF53A9000A1E0FE9000D6E0F418
:100DE800042EF53BE538B539058538378003120CF4
:100DF8001385372B752A008041E5379001D9126198
:100E08003CE0F538E5379001F912613CE0F539909E
:100E180000A1E0F404255EF53A9000B2E0FE9000EF
:100E2800A1E0F4042EF53BE538B53905853837805F
:100E380003120C1385372B752A00020EEC9000D98B
:100E4800E0D3955E5011E53790023912613CE0F528
:100E58002B752A00020EEC9000A2E0D3955E504359
:100E6800E53790021912613CE0F538E53790023910
:100E780012613CE0F5399000A2E0F404255EF53AF1
:100E88009000D9E0FE9000A2E0F4042EF53BE5388E
:100E9800B539058538378003120C1385372B752A29
:100EA800008041E5379001F912613CE0F538E537FB
:100EB80090021912613CE0F5399000B2E0F4042583
:100EC8005EF53A9000A2E0FE9000B2E0F4042EF540
:100ED8003BE538B539058538378003120C1385375B
:100EE8002B752A00229000EAE0F53C753F117559F0
:100EF80002755A00AE51AF52E53C75F00FA4FDAC37
:100F0800F0EDD39FEC9E4021E53C8E048F05FF1247
:100F180060FAED75F010A4FFAEF0E55E75F011848F
:100F2800FD7C00ED2FF53D800EE55E75F01184FF28
:100F38007E00EF24F0F53D853D37E55E75F01184C0
:100F4800AFF07E008F3A120B9985373EAE51AF5203
:100F58009000EAE075F00FA4FDACF0EDD39FEC9E95
:100F68004028755902755A10853D37120B99853EF0
:100F780038853739AE51AF52E53C8E048F05FF12E4
:100F880061258D3A853C3B120C138537297528005D
:100F9800752B64752A00229000EAE0F53C753F1134
:100FA800755902755A00AE51AF52E53C75F00FA461
:100FB800FDACF0EDD39FEC9E4021E53C8E048F05FF
:100FC800FF1260FAED75F010A4FFAEF0E56075F061
:100FD8001184FD7C00ED2FF53D800EE56075F01164
:100FE80084FF7E00EF24F0F53D853D37E56075F020
:100FF8001184AFF07E008F3A120B9985373EAE51BF
:10100800AF529000EAE075F00FA4FDACF0EDD39F6D
:10101800EC9E4028755902755A10853D37120B9978
:10102800853E38853739AE51AF52E53C8E048F0581
:10103800FF1261258D3A853C3B120C1385372975C3
:1010480028009000B4E0B40453E55E75F00484FF12
:101058007E008F37E55E75F00484ADF07C008D3A34
:10106800753F04755901755A00E537C3943F50051B
:10107800120B9980069001B8E0F537AE28AF29E544
:101088003712610A74648E048F05FF1260FAAE2865
:10109800AF29EF2DFDEE3CFC8C288D29752B64754E
:1010A8002A002290007FE0B40146E56675F00A84C4
:1010B800FF7E008F37E56675F00A84ADF07C008D01
:1010C8003A753F0A755905755A00E537C3941150AA
:1010D80005120B99800690058AE0F537AE2AAF2BEA
:1010E800E5372FFF50010E746412614E8E2A8F2B44
:1010F800900080E0B40146E56775F00A84FF7E0041
:101108008F37E56775F00A84ADF07C008D3A753F3E
:101118000A755905755A6CE537C394115005120BB9
:101128009980069005F6E0F537AE2AAF2BE5372F04
:10113800FF50010E746412614E8E2A8F2B90008F1F
:10114800E0B40249E569C3944175F00584FF7E0067
:101158008F37E56975F00584ADF07C008D3A753FF1
:1011680005755906755A00E537C394135005120BD7
:1011780099800690068CE0F537AE2AAF2BE5372F1D
:10118800FF50010E746412614E8E2A8F2B9000D18D
:10119800E0B40202800302124AE55E75F01584FF8E
:1011A8007E008F37E55E75F01584ADF07C008D3AD2
:1011B800753F15755903755AF4E537C3940B5005F7
:1011C800120B998006900478E0F537E53775F0FF43
:1011D800A4FFAEF09000D2E08E048F05FF1260FAF3
:1011E800ED90006BF0E56575F078A4FFAEF074FF44
:1011F8008E048F05FF1260FA8C598D5A74028C0682
:101208008D071200398F37AC59AD5A7404FF12613B
:10121800258D3A753F04755906755A28E537C394E4
:101228001D5005120B9980069006BEE0F537AE2AD0
:10123800AF2BE5372FFF50010E746412614E8E2AD2
:101248008F2B90007EE0B4025DE56075F064A4FF2A
:10125800AEF074081200398E5B8F5C74058E048FB3
:1012680005FF1260FA8D37AE5BAF5C74058E048F94
:1012780005FF1261258D3A753F05755905755ADECA
:10128800E537C394135005120B99800690066AE05F
:10129800F537AE2AAF2BE5372FFF50010E746412D5
:1012A800614E8E2A8F2B9000C0E0703C900047E082
:1012B80075F00584FF7E008F37900047E075F005D4
:1012C80084ADF07C008D3A753F05755905755AC097
:1012D800E537C3941D5005120B998006900656E019
:1012E800F537E537900073F022900087E0B40117D6
:1012F8009007C0E0252BFFAE2A50010E9000DBE0DE
:1013080012614E8E2A8F2B9000FFE0B401149001D9
:1013180000E0A851B8000495525007E55EC3955FF8
:10132800400280129000A9E0252BFFAE2A50010E42
:101338008E2A8F2B802F900087E0B40316A22EB33D
:10134800B350109007C3E0C39405A851B8000695A0
:1013580052400280109000A9E0252BFFAE2A5001D0
:101368000E8E2A8F2B900081E0B4020280030215B2
:101378004D900084E0602FE566D3944640289000A5
:1013880013E0FEA3E0FF9000BFE075F003A4FDACFE
:10139800F0EFD39DEE9C400E9000E3E0A851B8001A
:1013A80005D39552500302154D9000CCE0855EF0B0
:1013B800A4FFAEF0740512610A74071200398E5941
:1013C8008F5A90008BE0A851B800049552501290A3
:1013D800008CE075F002A4FDACF0EFC39DEE9C40DC
:1013E8000302154DE55E75F00B84FF7E009006093B
:1013F800126131FEE0FFEE900083E0FEEF8E008880
:10140800F0A4FFAEF074648E048F05FF1260FA8CAE
:10141800598D5A900047E075F018A4FFAEF090007F
:10142800CAE08E048F05FF1260FA8C068D079006BD
:1014380021126131AE59AF5AE012610A74648E0408
:101448008F05FF1260FA8C598D5AE564A859B800C7
:1014580077D3955A4072E564C3955AFFE49559FECF
:101468008E598F5A7428BE00039F500C755A2875E0
:101478005900740D900048F0AE59AF5A900084E0BE
:1014880012610A74288E048F05FF1260FA8C598D38
:101498005AAE28AF29740A8E048F05FF1260FA8DA0
:1014A800068C07AC59AD5ACFCECF120003740A8E02
:1014B800048F05FF1260FA8C598D5AAE28AF291295
:1014C80061568E288F29807DE564A859B800049557
:1014D8005A5072AE59AF5AE56412614E8E598F5AFE
:1014E8007428BE00039F500C755A28755900740D56
:1014F800900048F0AE59AF5A900084E012610A7427
:10150800288E048F05FF1260FA8C598D5AAE28AFC9
:1015180029740A8E048F05FF1260FA8D068C07ACB9
:1015280059AD5ACFCECF120003740A8E048F05FF2F
:101538001260FA8C598D5AAE28AF29EF2DFDEE3C7A
:10154800FC8C288D29229000DFE0B4026AE55E75E4
:10155800F00884FF7E008F37E55E75F00884ADF0F3
:101568007C008D3A753F08755901755AE0E537C317
:10157800943F5005120B998006900278E0F5378564
:10158800372D752C00AE2CAF2DAC2AAD2B120003D5
:1015980074648E048F05FF1260FA8C2C8D2D9000D8
:1015A8007CE08C068D0712610A74648E048F05FF37
:1015B8001260FA8C2C8D2DAE28AF29AC2AAD2B12D7
:1015C800000374648E048F05FF1260FA8C288D293D
:1015D80090007CE08C068D0712610A74648E048F7B
:1015E80005FF1260FA8C288D29A20D401DAE51AF5F
:1015F800527405BE00039F5002D20DE560D394CC0F
:101608004008D2017411900048F09000DEE0B40266
:10161800089000E0E0640160028035AE28AF29E55B
:101628006A12610A74E78E048F05FF1260FA8C282B
:101638008D299000DFE0B40217AE2CAF2DE56A12B9
:10164800610A74E78E048F05FF1260FA8C2C8D2DC9
:1016580090009EE05402601B900095E0A851B800ED
:1016680012D39552400DA20DB3B35007E560C39451
:101678009A40028028AE35AF36900093E075F002AC
:10168800A4FDACF0EF2DFDEE3CFC74022DFD5001E5
:101698000CE560BC0007D39D4003754301856036A7
:1016A800753500E54370030217919000F1E0C3958A
:1016B800435003021783900101E0C394025076E57A
:1016C8006675F00A84FF7E00900579126131E0F5B5
:1016D8005A755900AE59AF5A900094E012610A74D5
:1016E800648E048F05FF1260FA8C5B8D5C9000F1AC
:1016F800E004C395438C068D0712610A9000F1E05F
:101708008E048F05FF1260FA8C5B8D5CAE28AF29C2
:10171800EF2DFDEE3CFC8C288D299000DFE0B40213
:1017280012AE2CAF2DAA5BAB5CEF2BFBEE3AFA8A1C
:101738002C8B2D80469000F1E004C39543854BF037
:10174800A4FFAEF09000F1E08E048F05FF1260FA5E
:101758008C5B8D5CAE28AF29EF2DFDEE3CFC8C2810
:101768008D299000DFE0B40212AE2CAF2DAA5BAB3E
:101778005CEF2BFBEE3AFA8A2C8B2D05439000F197
:10178800E0C39543500375430090009EE054016008
:101798001B900092E0A851B80012D39552400DA2B8
:1017A8000DB3B35007E55EC394CC4002802590008A
:1017B80090E075F003A4FFAEF0E5402FFF50010E56
:1017C80074032FFF50010EE55EBE0007D39F400350
:1017D800754401855E40E54470030218C49000F228
:1017E800E0C3954450030218B6900101E0C3940287
:1017F8005076E56675F00A84FF7E009005791261DF
:1018080031E0F55A755900AE59AF5A900091E0127F
:10181800610A74648E048F05FF1260FA8C5B8D5C1C
:101828009000F2E004C395448C068D0712610A907B
:1018380000F2E08E048F05FF1260FA8C5B8D5CAEBF
:1018480028AF29EF2DFDEE3CFC8C288D299000DF78
:10185800E0B40212AE2CAF2DAA5BAB5CEF2BFBEE13
:101868003AFA8A2C8B2D80469000F2E004C3954406
:10187800854CF0A4FFAEF09000F2E08E048F05FFD7
:101888001260FA8C5B8D5CAE28AF29EF2DFDEE3C23
:10189800FC8C288D299000DFE0B40212AE2CAF2D0D
:1018A800AA5BAB5CEF2BFBEE3AFA8A2C8B2D054436
:1018B8009000F2E0C3954450037544009000F4E0B2
:1018C8002529FFAE2850010E8E288F299000A3E00D
:1018D800A828B80004952950099000A3E0F52975B7
:1018E80028009000DFE0B4020D9000A3E0A82CB817
:1018F8000006952D400280099000A3E0F52D752C77
:1019080000229000DFE0B401028003021A15A20D44
:10191800B35003021A139000AAE0B40168AE28AFCE
:1019280029AC51AD52120003743C8E048F05FF128E
:1019380060FA9000BAE0BC00109D400D9000BCE039
:10194800A828B8000495295002D202AE28AF29ACC5
:1019580051AD52120003743C8E048F05FF1260FAD9
:101968009000BAE0C3940ABC0015D39D40119000C2
:10197800BCE0C39405A828B80005D3952950028077
:1019880002C2028068AE28AF29AC51AD52120003E2
:1019980074788E048F05FF1260FA9000BAE0BC00DC
:1019A800109D400D9000BCE0A828B800049529506F
:1019B80004D2028038AE28AF29AC51AD52120003D0
:1019C80074788E048F05FF1260FA9000BAE0C39411
:1019D8000ABC0015D39D40119000BCE0C39405A833
:1019E80028B80005D3952950028002C202A202B38A
:1019F8004019AE28AF299000BBE012610A74648ECA
:101A0800048F05FF1260FA8C288D298002C202A279
:101A180000B34006A201B3B35009900019E4F0A343
:101A2800F08024AE28AF297400D39F74019E400C27
:101A3800900019E528F0A3E529F0800B74FF9000C9
:101A480019F8E4F0E8A3F09000C1E0D39402400C48
:101A58009000ACE07006A20DB3B34002801AAE2825
:101A6800AF29740212610A8E288F29AE2CAF2D740B
:101A78000212610A8E2C8F2D9000AAE0B4011AAED2
:101A880028AF29740212610A8E288F29AE2CAF2D37
:101A9800740212610A8E2C8F2DAE28AF29745E1243
:101AA800610A740A8E048F05FF1260FA8C288D294A
:101AB8009000DFE0B40217AE2CAF2D745E12610AFD
:101AC800740A8E048F05FF1260FA8C2C8D2DAE28B7
:101AD800AF297402BE000AD39F40067529027528F3
:101AE80000AE2CAF2D7402BE000AD39F4006752DA0
:101AF80002752C00900017E528F0A3E529F0229044
:101B08000047E090037912613CE0F541754264902A
:101B18000047E0FE9000B5E0D39E4037E55E75F0E3
:101B28000884FF7E008F37E55E75F00884ADF07C91
:101B3800008D3A753F08755903755A96E537C39471
:101B48001F5005120B99800690042EE0F537853753
:101B5800428035E55E75F00884FF7E008F37E55ECC
:101B680075F00884ADF07C008D3A753F087559030F
:101B7800755AB6E537C3941F5005120B9980069025
:101B8800044EE0F537853742229000EBE0F53C75CE
:101B98003F11755904755A00AE51AF52E53C75F0C6
:101BA8000FA4FDACF0EDD39FEC9E4021E53C8E04E4
:101BB8008F05FF1260FAED75F010A4FFAEF0E55E38
:101BC80075F01184FD7C00ED2FF53D800EE55E7506
:101BD800F01184FF7E00EF24F0F53D853D37E55E8A
:101BE80075F01184AFF07E008F3A120B9985373E5D
:101BF800AE51AF529000EBE075F00FA4FDACF0EDE4
:101C0800D39FEC9E4028755904755A10853D3712AC
:101C18000B99853E38853739AE51AF52E53C8E0475
:101C28008F05FF1261258D3A853C3B120C138537D1
:101C380041754264229000EBE0F53C753F117559FF
:101C480004755A00AE51AF52E53C75F00FA4FDACD7
:101C5800F0EDD39FEC9E4021E53C8E048F05FF12EA
:101C680060FAED75F010A4FFAEF0E56075F0118430
:101C7800FD7C00ED2FF53D800EE56075F01184FFC9
:101C88007E00EF24F0F53D853D37E56075F0118461
:101C9800AFF07E008F3A120B9985373EAE51AF52A6
:101CA8009000EBE075F00FA4FDACF0EDD39FEC9E37
:101CB8004028755904755A10853D37120B99853E91
:101CC80038853739AE51AF52E53C8E048F05FF1287
:101CD80061258D3A853C3B120C138537417542646A
:101CE8009000E6E0B40479900047E0FE9000B5E08B
:101CF800D39E4037E55E75F00884FF7E008F37E598
:101D08005E75F00884ADF07C008D3A753F08755912
:101D180003755A96E537C3941F5005120B99800630
:101D280090042EE0F5378537428035E55E75F0087A
:101D380084FF7E008F37E55E75F00884ADF07C0087
:101D48008D3A753F08755903755AB6E537C3941F20
:101D58005005120B99800690044EE0F537853742FE
:101D68002290007FE0B4013BE56675F00A84FF7EAF
:101D7800008F37E56675F00A84ADF07C008D3A7502
:101D88003F0A755905755A12E537C3941150051263
:101D98000B99800690059CE0F537E5422537C394FA
:101DA80064F542900080E0B4013BE56775F00A8471
:101DB800FF7E008F37E56775F00A84ADF07C008DF3
:101DC8003A753F0A755905755A7EE537C39411501F
:101DD80005120B998006900608E0F537E54225378D
:101DE800C39464F542E5412542F534900087E0B498
:101DF80002109007BFE02534FE9000DBE0F4042ECB
:101E0800F5349000DEE0D394014040E56AC394E7DE
:101E1800501D74E7C3956AFE9007C1E08E00F5F087
:101E2800E884FF7E008F37E5342537F534801CE5DC
:101E38006AC394E7FE9007C1E08E00F5F0E884FFDE
:101E48007E008F37E534C39537F534A20D4006E59B
:101E5800412464F534E534D394644009E534C394EB
:101E680064F53480037534009000B7E0C3953450AE
:101E7800069000B7E0F53422D200900071E0A85136
:101E8800B8000495525041900071E0A851B8000480
:101E98009552500375340F900071E004A851B800B2
:101EA800049552500375340A900071E02402A85139
:101EB800B8000495525005753405C200900071E0D1
:101EC80060067409900048F0C23E7E017F009000D1
:101ED800BDE012610A9000CCE08E048F05FF12600D
:101EE800FAE55EBC0017D39D40139000C6E0B4022B
:101EF80004D23E8002C200740A900048F09000BEEE
:101F0800E0C3956650159000D0E0A851B80004953C
:101F1800525002C200740B900048F0E566C3946406
:101F2800501D900116E0600D900116E0A851B80010
:101F380006955240028008C200740B900048F0A237
:101F48000040037534059000FFE0B40114900100CF
:101F5800E0A851B8000495525007E55EC3955F406C
:101F68000280089000A8E0F534803A900087E0B439
:101F78000306A22EB3B34002802B9007C3E0C3949C
:101F880005A851B800049552500C9000A8E0F5340B
:101F9800740C900048F09007C3E0A851B80004956D
:101FA800525002C20085346B900079E02534FE90CF
:101FB8000047E075F01E84FC7F00EE2CF53422907B
:101FC8000047E075F00584FF7E008F37900047E0FA
:101FD80075F00584ADF07C008D3A753F05755903A1
:101FE800755AD69000CAE01475F00584FF7E00E5A6
:101FF80037BE00039F5005120B99800BE5379004FC
:102008004F12613CE0F537E5379007C2F09007C200
:10201800E0FE9000B9E0C39E50089000B9E0900738
:10202800C2F022E56675F00A84FF7E0090057912F9
:102038006131E0F546E546D394644010E546C39423
:102048006475F00F84FF7E008F468003754600900C
:10205800009CE02546F546229007B3E0FEA3E0FF8A
:102068007404120039E55E12610A740F8E048F053C
:10207800FF1260FA9007B1ECF0A3EDF090008FE04A
:10208800B40262E569C3944175F00584FF7E008F50
:1020980037E56975F00584ADF07C008D3A753F052C
:1020A800755906755A14E537C394175005120B99DC
:1020B80080069006A0E0F5379007B1E0FEA3E0FFA8
:1020C800740A8E048F05FF1260FAE5378C068D07B7
:1020D80012610A740A8E048F05FF1260FA9007B124
:1020E800ECF0A3EDF09007B1E0FEA3E0FF9007B796
:1020F800E0FCA3E0FDEDD39FEC9E400F9007B7E016
:10210800F8A3E09007B1C8F0A3C8F0229006C0E099
:10211800903419F8282873804C85527280479000B3
:10212800CCE0855EF0A4FFAEF074081200398F721F
:102138008033856072802E856672802985677280FB
:1021480024856872801F856972801A856A72801575
:102158008565728010856472800B856B728006902D
:05216800001AE0F57211
:1034190002211F02212102212602213A02213F0213
:10342900214402214902214E02215302215802213D
:073439005D02216202216720
:10216D009006C1E0FE9006C2E0D39E404B9006C0A3
:10217D00E0B404189006C2E0C395725002D22F90BD
:10218D0006C1E0D395724002C22F802A9006C1E0AD
:10219D00C3957250099006C2E0D395725002800229
:1021AD00D22F9006C1E0D3957250099006C2E0C3BC
:1021BD0095725002C22F802A9006C1E0D3957240CD
:1021CD00099006C2E0C3957240028002C22F9006AC
:1021DD00C1E0C3957240099006C2E0D395724002EA
:1021ED00D22F229006C4E0903440F8282873804CFA
:1021FD0085527280479000CCE0855EF0A4FFAEF072
:10220D0074081200398F728033856072802E856656
:10221D007280298567728024856872801F85697236
:10222D00801A856A7280158565728010856472804A
:0C223D000B856B72800690001AE0F572B1
:103440000221FB0221FD02220202221602221B029D
:10345000222002222502222A02222F0222340222C4
:073460003902223E02224363
:102249009006C5E0FE9006C6E0D39E405F9006C4A6
:10225900E0B404189006C6E0C395725002D23090DB
:1022690006C5E0D395724002C230803E9006C5E0B3
:10227900C3957250099006C6E0D395725002800248
:10228900D2309006C5E0D3957250099006C6E0C3D6
:1022990095725002C2309006C4E0B401099000D88A
:1022A900E0D3956050028002C230802A9006C5E0D2
:1022B900D3957240099006C6E0C395724002800228
:1022C900C2309006C5E0C3957240099006C6E0D3B6
:1022D90095724002D230229006C8E0903467F828FF
:1022E9002873804C85527280479000CCE0855EF05F
:1022F900A4FFAEF074081200398F728033856072C2
:10230900802E85667280298567728024856872802F
:102319001F856972801A856A7280158565728010B9
:10232900856472800B856B72800690001AE0F572E5
:103467000222EB0222ED0222F202230602230B02C2
:10347700231002231502231A02231F0223240223E7
:073487002902232E0223336A
:102339009006C9E0FE9006CAE0D39E404B9006C8BD
:10234900E0B404189006CAE0C395725002D23190E5
:1023590006C9E0D395724002C231802A9006C9E0CD
:10236900C3957250099006CAE0D395725002800253
:10237900D2319006C9E0D3957250099006CAE0C3DC
:1023890095725002C231802A9006C9E0D3957240F5
:10239900099006CAE0C3957240028002C2319006D4
:1023A900C9E0C3957240099006CAE0D3957240020C
:1023B900D231229006CCE090348EF8282873804CD4
:1023C90085527280479000CCE0855EF0A4FFAEF0A4
:1023D90074081200398F728033856072802E856689
:1023E9007280298567728024856872801F85697269
:1023F900801A856A7280158565728010856472807D
:0C2409000B856B72800690001AE0F572E3
:10348E000223C70223C90223CE0223E20223E7024C
:10349E0023EC0223F10223F60223FB022400022472
:0734AE000502240A02240FAD
:102415009006CDE0FE9006CEE0D39E404B9006CCD4
:10242500E0B404189006CEE0C395725002D2329003
:1024350006CDE0D395724002C232802A9006CDE0E7
:10244500C3957250099006CEE0D395725002800272
:10245500D2329006CDE0D3957250099006CEE0C3F6
:1024650095725002C232802A9006CDE0D395724013
:10247500099006CEE0C3957240028002C2329006F2
:10248500CDE0C3957240099006CEE0D39572400227
:10249500D232229006D0E09034B5F8282873804CCB
:1024A50085527280479000CCE0855EF0A4FFAEF0C7
:1024B50074081200398F728033856072802E8566AC
:1024C5007280298567728024856872801F8569728C
:1024D500801A856A728015856572801085647280A0
:0C24E5000B856B72800690001AE0F57207
:1034B5000224A30224A50224AA0224BE0224C302D4
:1034C50024C80224CD0224D20224D70224DC0224FB
:0734D500E10224E60224EBF2
:1024F1009006D1E0FE9006D2E0D39E404B9006D0EC
:10250100E0B404189006D2E0C395725002D2339021
:1025110006D1E0D395724002C233802A9006D1E001
:10252100C3957250099006D2E0D395725002800291
:10253100D2339006D1E0D3957250099006D2E0C310
:1025410095725002C233802A9006D1E0D395724031
:10255100099006D2E0C3957240028002C233900610
:10256100D1E0C3957240099006D2E0D39572400242
:10257100D233229006D4E09034DCF8282873804CC2
:1025810085527280479000CCE0855EF0A4FFAEF0EA
:1025910074081200398F728033856072802E8566CF
:1025A1007280298567728024856872801F856972AF
:1025B100801A856A728015856572801085647280C3
:0C25C1000B856B72800690001AE0F5722A
:1034DC0002257F02258102258602259A02259F025C
:1034EC0025A40225A90225AE0225B30225B8022582
:0734FC00BD0225C20225C735
:1025CD009006D5E0FE9006D6E0D39E404B9006D403
:1025DD00E0B404189006D6E0C395725002D2349040
:1025ED0006D5E0D395724002C234802A9006D5E01C
:1025FD00C3957250099006D6E0D3957250028002B1
:10260D00D2349006D5E0D3957250099006D6E0C32A
:10261D0095725002C234802A9006D5E0D39572404F
:10262D00099006D6E0C3957240028002C23490062E
:10263D00D5E0C3957240099006D6E0D3957240025D
:10264D00D234229006D8E0903503F8282873804CB8
:10265D0085527280479000CCE0855EF0A4FFAEF00D
:10266D0074081200398F728033856072802E8566F2
:10267D007280298567728024856872801F856972D2
:10268D00801A856A728015856572801085647280E6
:0C269D000B856B72800690001AE0F5724D
:1035030002265B02265D02266202267602267B02E3
:10351300268002268502268A02268F022694022608
:073523009902269E0226A377
:1026A9009006D9E0FE9006DAE0D39E404B9006D81A
:1026B900E0B404189006DAE0C395725002D235905E
:1026C90006D9E0D395724002C235802A9006D9E036
:1026D900C3957250099006DAE0D3957250028002D0
:1026E900D2359006D9E0D3957250099006DAE0C345
:1026F90095725002C235802A9006D9E0D39572406E
:10270900099006DAE0C3957240028002C23590064C
:10271900D9E0C3957240099006DAE0D39572400278
:10272900D235229006DCE090352AF8282873804CAF
:1027390085527280479000CCE0855EF0A4FFAEF030
:1027490074081200398F728033856072802E856615
:102759007280298567728024856872801F856972F5
:10276900801A856A72801585657280108564728009
:0C2779000B856B72800690001AE0F57270
:10352A0002273702273902273E022752022757026B
:10353A00275C02276102276602276B02277002278F
:07354A007502277A02277FBA
:102785009006DDE0FE9006DEE0D39E404B9006DC31
:10279500E0B404189006DEE0C395725002D236907C
:1027A50006DDE0D395724002C236802A9006DDE050
:1027B500C3957250099006DEE0D3957250028002EF
:1027C500D2369006DDE0D3957250099006DEE0C35F
:1027D50095725002C236802A9006DDE0D39572408C
:1027E500099006DEE0C3957240028002C23690066B
:1027F500DDE0C3957240099006DEE0D39572400294
:10280500D236229006E0E0903551F8282873804CA6
:1028150085527280479000CCE0855EF0A4FFAEF053
:1028250074081200398F728033856072802E856638
:102835007280298567728024856872801F85697218
:10284500801A856A7280158565728010856472802C
:0C2855000B856B72800690001AE0F57293
:1035510002281302281502281A02282E02283302F3
:10356100283802283D02284202284702284C022816
:073571005102285602285BFD
:102861009006E1E0FE9006E2E0D39E404B9006E048
:10287100E0B404189006E2E0C395725002D237909A
:1028810006E1E0D395724002C237802A9006E1E06A
:10289100C3957250099006E2E0D39572500280020E
:1028A100D2379006E1E0D3957250099006E2E0C379
:1028B10095725002C237802A9006E1E0D3957240AA
:1028C100099006E2E0C3957240028002C237900689
:1028D100E1E0C3957240099006E2E0D395724002AF
:1028E100D237229006E4E0903578F8282873804C9E
:1028F10085527280479000CCE0855EF0A4FFAEF077
:1029010074081200398F728033856072802E85665B
:102911007280298567728024856872801F8569723B
:10292100801A856A7280158565728010856472804F
:0C2931000B856B72800690001AE0F572B6
:103578000228EF0228F10228F602290A02290F027E
:10358800291402291902291E02292302292802299D
:073598002D02293202293740
:10293D009006E5E0FE9006E6E0D39E404B9006E45F
:10294D00E0B404189006E6E0C395725002D23890B8
:10295D0006E5E0D395724002C238802A9006E5E084
:10296D00C3957250099006E6E0D39572500280022D
:10297D00D2389006E5E0D3957250099006E6E0C393
:10298D0095725002C238802A9006E5E0D3957240C8
:10299D00099006E6E0C3957240028002C2389006A7
:1029AD00E5E0C3957240099006E6E0D395724002CA
:1029BD00D23822AE2EAF2F74F5D39F74019E4008EE
:1029CD00782E12615E022ADA752F01752E00AE5136
:1029DD00AF52E546BE000DD39F40099000AEE0D347
:1029ED00954740028023754700E546C39552F57221
:1029FD009000B1E0D395454008E5452572F5458039
:102A0D00069000B1E0F5458002054790008AE0D3BD
:102A1D009560401CE55EC3955F4015AE51AF52E524
:102A2D0046BE00039F50099000AFE0D39548400289
:102A3D00806E9007C6E0A851B800049552500375FA
:102A4D004A009007C6E0A851B8000BD39552400636
:102A5D00E5529007C6F0E54A7041E552C39546F53B
:102A6D0072E572D3940540037572059000B0E0C312
:102A7D0095455007E572C3954540028009E545C36C
:102A8D009572F54580069000B0E0F5459000B0E0F8
:102A9D00D3954540069000B0E0F54575480080029D
:102AAD000548E54A701690008AE0C39560500DE523
:102ABD00462405A851B8000695524002800F90009B
:102ACD009DE0F545754A0174789007C6F022AE2E4B
:102ADD00AF2F74E9D39F74039E4008782E12615E68
:102AED00022C79752F01752E00754532A239402AB9
:102AFD0075451990009DE075F002A4FFAEF0E54715
:102B0D00BE0006D39F4002D2390547754A0374783B
:102B1D009007C6F0754900022C68AE51AF52E546DC
:102B2D006F4E7003022C68E546BE000DD39F400921
:102B3D009000AEE0D395474002800F754700E54AFF
:102B4D00C394035003754519800DE546C39552F5A1
:102B5D0072E5472572F54790008AE0D39560400EE7
:102B6D009007C6E0A851B80007D395524002800CDB
:102B7D00054990009DE0B54903754A00E54AB40347
:102B8D0006A20DB3B34002800A0549E549B43C03E2
:102B9D00754A02E54AB402299007C6E0A851B8006B
:102BAD000ED395524009E5529007C6F07549009035
:102BBD00008AE0C39560500975490074789007C686
:102BCD00F0E54A705A90008AE0D39560401CE55EAE
:102BDD00C3955F4015AE51AF52E546BE00039F5001
:102BED00099000AFE0D39548400280087548007504
:102BFD00454B8028E552C39546F572E572D3940591
:102C0D00400375720590008AE0D395604008E54851
:102C1D002572F5488006E5482406F548754900E516
:102C2D004A701690008AE0C39560500DE546240564
:102C3D00A851B80006955240028003754A01E54A35
:102C4D00B40118754519054990009DE0B549067503
:102C5D004A0275490074789007C6F0E54575F00A8B
:102C6D00A4FFAEF09007BBEEF0A3EFF022E56E905F
:102C7D00359FF8282873900082E07003022E28906B
:102C8D0000B8E0B401028003022D78900046E0B553
:102C9D005D028003022D757E017F00E5BE12610A83
:102CAD00E5BD2FFF50010E8E598F5A741012610A17
:102CBD00900070E08E048F05FF1260FA9007C7EC4C
:102CCD00F0A3EDF0E56A60089000DEE064026002BA
:102CDD0080269000E0E0B4011F9007C7E0FEA3E05E
:102CED00FF74E712610AE56A8E048F05FF1260FA20
:102CFD009007C7ECF0A3EDF0900082E0B4022790AE
:102D0D0007C9E0FEA3E0FF9007C7E0FCA3E0FDEFDD
:102D1D002DFDEE3CFC74018C068D071200399007D9
:102D2D00C7EEF0A3EFF09007C7E0FEA3E0FF90071A
:102D3D00C9E0FCA3E0FDEDD39FEC9E4004D23C80A6
:102D4D0002B23C9007C7E0F8A3E09007C9C8F0A312
:102D5D00C8F09000B4E064016006A23CB3B3400239
:102D6D0080069007C8E0F55E022E26D23C7E017FDC
:102D7D0000E5BE12610AE5BD2FFF50010E8E598F81
:102D8D005A741012610A900070E08E048F05FF12C4
:102D9D0060FA9007C7ECF0A3EDF0E56A60089000CB
:102DAD00DEE06402600280269000E0E0B4011F9036
:102DBD0007C7E0FEA3E0FF74E712610AE56A8E041F
:102DCD008F05FF1260FA9007C7ECF0A3EDF09000AD
:102DDD0082E0B402279007C9E0FEA3E0FF9007C789
:102DED00E0FCA3E0FDEF2DFDEE3CFC74018C068DA7
:102DFD00071200399007C7EEF0A3EFF09007C7E078
:102E0D00F8A3E09007C9C8F0A3C8F09000B4E0643F
:102E1D000160069007C8E0F55E8003755E009000C6
:102E2D007EE07006756E01022C7A75BB180233F3C5
:102E3D0090007EE07003022FC97E017F00E5BE1277
:102E4D00610AE5BD2FFF50010E8E598F5A9000C4B7
:102E5D00E0B4010F7E0F7FFFAC59AD5A1261568E53
:102E6D00598F5A9000E9E0B40245AE59AF5A90001F
:102E7D0023E0FCA3E0FDEDD39FEC9E400A900023E0
:102E8D00E559F0A3E55AF0AE59AF5A900025E0FC94
:102E9D00A3E0FDEFD39DEE9C400A900025E559F08F
:102EAD00A3E55AF0AE59AF5A74041200398F6090F1
:102EBD0000E9E0704CAE59AF5A900023E0FCA3E05E
:102ECD00FDEFD39DEE9C40091261568E598F5A80AD
:102EDD0006755A00755900AE59AF5A741012610A31
:102EED0090006DE08E048F05FF1260FA8C598D5A9B
:102EFD0074FFBC0009D39D4005855A608003756041
:102F0D00FE9000B4E0B401028003022FC7A20DB3FE
:102F1D00B3500E900088E0A851B80005D3955250DB
:102F2D0003022FBC900089E075F019A4FFAEF0905C
:102F3D0000CCE08E048F05FF1260FA9000C5E0858D
:102F4D0060F0A4FFAEF074648D028C038E048F05C7
:102F5D00FF1260FAEA2DFDEB3CFC8C598D5AE56AA7
:102F6D00600F9000DEE0B402089000E0E0640160C4
:102F7D00028017AE59AF5A74E712610AE56A8E04E2
:102F8D008F05FF1260FA8C598D5AAE59AF5A9007C2
:102F9D00C7E0FCA3E0FDEDD39FEC9E4005855A5E96
:102FAD00800BA23CB340069007C8E0F55E800BA2F3
:102FBD003CB340069007C8E0F55E80037560009055
:102FCD000081E07006756E02022C7A75BB19023312
:102FDD00F3900081E0700302307EE55DD3955040A3
:102FED000302307C900021E0FEA3E0FFE564126156
:102FFD004E900021EEF0A3EFF07E017F00E5BE12B2
:10300D00610AE5BD2FFF50010E8E598F5A9000EECB
:10301D00E07013740A12610A74518E048F05FF1249
:10302D0060FA8D648019AE59AF5A740A12610A8F15
:10303D00048E057E017F95CDCCCD125FF88F64E5B2
:10304D0064D394644003756464900021E0FEA3E0B2
:10305D00FFE5642FFF50010E900021EEF0A3EFF07D
:10306D00900085E0048E048F05FF1260FA8D648058
:10307D00037564329000D1E07006756E03022C7AF0
:10308D0075BB130233F39000D1E0604A7E017F00DF
:10309D00E5BE12610AE5BD2FFF50010E8E598F5A04
:1030AD0074041200398F659000D3E08565F0A4FD9E
:1030BD00ACF07464FF1260FA8D659000D2E0856506
:1030CD00F0A4FFAEF074FF8E048F05FF1260FAEDD1
:1030DD0090006CF0800375650090007FE0700675C0
:1030ED006E04022C7A75BB170233F390007FE0B4A7
:1030FD000102800302318C7E017F00E5BE12610A60
:10310D00E5BD2FFF50010E8E598F5A9007CBE06011
:10311D00199007CBE014905A7612008CE493FC744E
:10312D000193FDEDC39FEC9E400280069007CBE01E
:10313D0014F09007CBE0C394B3501DAE59AF5A9025
:10314D0007CBE004905A7612008CE493FC74019343
:10315D00FDEFC39DEE9C400280069007CBE004F08E
:10316D009007CBE0FE9000A5E08E0088F0A4FFAEA6
:10317D00F074648E048F05FF1260FA8D66800375FE
:10318D006600900080E07006756E05022C7A75BBA6
:10319D00160233F3900080E0B40102800302323551
:1031AD007E017F00E5BE12610AE5BD2FFF50010EC5
:1031BD008E598F5A9007CCE060199007CCE014908F
:1031CD005BE012008CE493FC740193FDEDC39FEC66
:1031DD009E400280069007CCE014F09007CCE0C32F
:1031ED0094B3501DAE59AF5A9007CCE004905BE0FC
:1031FD0012008CE493FC740193FDEFC39DEE9C4093
:10320D000280069007CCE004F09007CCE0FE900021
:10321D00ABE08E0088F0A4FFAEF074648E048F05D1
:10322D00FF1260FA8D67800375670075BB1F02334F
:10323D00F37E017F00E5BE12610AE5BD2FFF50014F
:10324D000E8E598F5A740912610A74E68E048F0519
:10325D00FF1260FA8D69900087E07006756E0702A7
:10326D002C7A75BB150233F3900087E0700302339F
:10327D008F7E017F00E5BE12610AE5BD2FFF500173
:10328D000E8E598F5A74041200398F68900087E0A2
:10329D00B401159000DBE08568F0A4FFAEF0740773
:1032AD00120039EF9007C0F0900087E0B40215903E
:1032BD0000DBE08568F0A4FFAEF07407120039EF73
:1032CD009007BFF0900087E0B40302800302338DB6
:1032DD009000C8E070389000DBE0601CE568C39496
:1032ED00195002D22EE568D394644002C22E90008C
:1032FD00A7E09007C3F08014E568C394195002D27B
:10330D003DE568D394324002C23DC22E80639000E9
:10331D00A7E070349000DBE08568F0A4FFAEF07498
:10332D00FF8E048F05FF1260FAED9007C3F0AE51CA
:10333D00AF52741EBE0006D39F4002D22EE560D35D
:10334D0094E54002C22E8029E568C3940A500DAE63
:10335D0051AF52741EBE0004D39F50028002D22E74
:10336D00E560D394E54002C22E9000A7E09007C31C
:10337D00F09007C3E0C39405500674059007C3F0A1
:10338D0080037568009000DEE07006756E08022CF3
:10339D007A75BB1480509000DEE060397E017F00AD
:1033AD00E5BE12610AE5BD2FFF50010E8E598F5AF1
:1033BD00EFD39421EE940E4005756AFF8015AE593A
:1033CD00AF5A741012610A74E38E048F05FF1260F8
:1033DD00FA8D6A8003756A00900082E0600575BB06
:0633ED001A800375BB18F5
:10359F00022C83022E3D022FDE0230930230F802FE
:0B35AF0031A102323E0232750233A34C
:0533F300056ED2EC2282
:09613C002582F582500205832240
:0F008C0025E050020583258250020583F582226C
:1060D900EF2F500205832582F582E5833E2EF58355
:0160E9002294
:10614E00CFC39FFF50011E22C3EF9DFFEE9CFE2288
:08615E000806B6000218062233
:0D611800A3E004F07006120049E004F0223C
:0E003900048007C3CE13CECF13CFD5E0F6223E
:105FF800BC000FBE0008ED8FF084FFADF022E4FE78
:10600800FF22BE000DEF60FE54F0606F20E7030230
:1060180060AEEAC0E0EBC0E078017A0075F001EE0E
:1060280020E710EF25E0FFEE33FE0AC5F023C5F0A8
:1060380030E7F0EA5407F9096A7A007B0060010842
:10604800C3EC9E40167004ED9F4010ED9FFDEC9E42
:10605800FCE5F0CA4ACA03F5F08005E5F003F5F05F
:10606800C3EE13FEEF13FFD9D77908CACBCAD8D02D
:10607800EAFEEBFFD0E0FBD0E0FA22EC8FF084FCE4
:10608800ED54F045F0C48FF084FEEDC454F045F0B3
:10609800C48FF084FDEEC4FE54F02DFFEE540F3C87
:1060A800FEADF07C0022790078008FF0EC7E0820AD
:1060B800E70DC3CD33CD33C933C9C833C8DEF08447
:1060C80049F9E5F08FF0BE00E6FD7C00E9FFE8FE47
:0160D80022A5
:0E610A00F88FF0A4FFE5F0CE88F0A42EFE2260
:10000300EF8DF0A4F9A8F0EF8CF0A428F8EE8DF0B2
:06001300A428FEE9FF2213
:1060EA00600D782B0260F4007830D8FED5E0F822F3
:1060FA00EEC0E07E00125FF8EFFDEEFCD0E0FE227B
:0C612500EEC0E07E00125FF8D0E0FE2229
:03001B0002001EC2
:0300530002005652
:03009B00020071EF
:0300000002614555
:0961450075817475D000023DCB98
:0B613100E5822FF582E5833EF5832216
:0A0049000582D5820215831582227C
:10001E00C0E0C0F0C083C082C0D075D000123D37A2
:0B002E00D0D0D082D083D0F0D0E032E0
:10005600C0E0C0F0C083C082C0D075D000123D3A67
:10006600D0D0D082D083D0F0D0E032C0E0C0F0C093
:1000760083C082C0D075D000123D56D0D0D082D079
:0600860083D0F0D0E0324F
:00000001FF
